:100000006E28FF3FFF3FFF3FDF00030E8301AF007D
:100010000408AE000A08B0008A015008B3000B11B2
:10002000200803191428A003A10A2108113C031871
:100030001A28A101A20A2208113C03182028A201B3
:10004000A30A2308113C03182628A301240821022F
:1000500003182C2885142D28851025082202031842
:1000600033280514342805102608230203183A28DB
:1000700005153B2805113308D00030088A002E08EA
:1000800084002F0E8300DF0E5F0E0900031383121E
:10009000A401A501A6010130A700080003138312E3
:1000A000320883169B009C131C141A08D000080009
:1000B000031383122808A4002908A5002A08A60013
:1000C0000430A7000800031383122B08A4002C0897
:1000D000A5002D08A6000230A7000800C8300313B1
:1000E0008312A000073099003830831685005830FD
:1000F0009F000D3083129F00A0308B00D0308316FC
:1001000081008312851005100511A1010630A2009F
:100110000C30A30046204B30B1009F14B2014E209A
:100120005008AB000130B2004E205008AC00023045
:10013000B2004E205008AD000330B2004E205008EF
:10014000A8000430B2004E205008A9000530B200CB
:100150004E205008AA0083129F18F0282008031D83
:10016000F0281E0831020318B728B10ABC2831084C
:100170001E020318BC28B103E12831087D3C031896
:10018000C3285820C8283108323C0318C8286320E7
:10019000ED2831087D3C0318CF285820D428193089
:1001A00031020318D4284620ED28193031020318F3
:1001B000DB284620E028643031020318E028632061
:1001C000ED282708013A0319BD282708023A031928
:1001D000C9282708043A0319D5289F140230A00023
:1001E000AB28F128FF3FFF3FFF3FFF3FFF3FFF3FAF
:02400E00D43F9D
:00000001FF
